:10000000031E080086015F308C000D3084008001E3
:10001000840A8C0B07282C282120840007398406A9
:100020000310840C840C840C041A841704128A01B3
:10003000820701340234043408341034203440344C
:10004000803407398A018207303431343234333412
:1000500034343534363437348030A20086301F22B1
:100060000430142204215721900100308A00100826
:10007000F33E03184D280D3E3F208E004D28820789
:10008000503472346F346734723461346D342034D8
:100090006234793420342D342034722110089122B6
:1000A0006B222208900000308122031D5B280C3057
:1000B000772203193528C0308E0059219001003075
:1000C0008A001008F03E03187A28103E69208E003E
:1000D0007A28820754346534633468345F34533487
:1000E000633469342034263420344E344534453466
:1000F0004C3442347221100891226B222208900065
:1001000000308122031D88280F30772203195F28D1
:1001100037309422912201307C22031D90288828B8
:1001200037309422912200307C22031D9828902899
:100130005721900100308A001008EE3E0318B728BE
:10014000123EA4208E00B7288207533465346C34E5
:1001500066345F34743465347334743469346E34A3
:1001600067342E342E342E342E342E342E34722115
:10017000100891226B222208900000308122031D7A
:10018000C5280F30772203199A28C8302322572117
:1001900037309422912201307C22031DD028C828B8
:1001A00037309422912200307C22031DD828D02899
:1001B00007309C22A801D4218E003730942291224E
:1001C00001307C22031DE528DD280E0891228030B5
:1001D0007722031DC1290E08912201307C22031DC4
:1001E0003E290E08912202307C22031D29290E0887
:1001F000912203307C22031D30290E089122043005
:100200007C22031D37299729143023220330A200B2
:1002100006301F22C821053023220330A2000630F9
:100220001F22C821013023220330A20006301F22E2
:10023000C821013023220230A20006301F22C8212B
:1002400028308E0059210C308E00592106308E0046
:1002500059290E089122BE305B2222088E003E29C9
:100260000E08912211305B2222088E003E290E08D2
:10027000912209305B2222088E003E290E0891222D
:100280001030392222088F000F08A20006301F22EA
:10029000C8210E0891220F30502222088F000F082B
:1002A000A20006301F22C82101302322C8280130B5
:1002B0008E000E0891221030392222088F000F087C
:1002C000A20006301F22C8210E0891220F305022B2
:1002D00022088F000F08A20006301F22C82101301B
:1002E0002322A12A0E0891221030392222088F00E1
:1002F0000F08912220305B2222088F000F08A200F5
:1003000006301F22C8210E0891220F3050222208E9
:100310008F000F08912220305B2222088F000F08E7
:10032000A20006301F22C82101302322A12A0E0874
:1003300091221030392222088F000F08912220309C
:100340005B2222088F000F08A20006301F22013016
:100350002322C8210E0891220F30502222088F003C
:100360000F08912220305B2222088F000F08A20084
:1003700006301F2201302322C821013023228E01A2
:10038000C8280E0891228030572222088E00E528C6
:100390000430182201302322043014220130232299
:1003A000A12A07303122D129270884008417260882
:1003B00080046400E8210318D929F2210830AA003A
:1003C000F421E821AB0CAA0BE029F4212B0808004A
:1003D0002708840026080005281926060310031D97
:1003E000031408002817FB290330F7290230FF3EC9
:1003F000031DF729281302308A00280D06398207C9
:100400000830082A1030082A0230082A4030082A0A
:10041000A900281BA90C112A0C30FF3E031D0D2A30
:100420000000A90B0C2A08000C20FF3A80051C2AAA
:100430000C2080041B2AFF3A84178005A12A84001F
:1004400022088000A12AA301A200692264002308D7
:10045000220403190800F730FF3E031D2C2A6B22EB
:10046000262A83160739F83881006300FF3081009F
:10047000A12AA501A4001030AB00AA01A901031410
:10048000A20DA30DA90DAA0D6F2229305E22031C17
:1004900022106F222930221C5E22AB0B3F2AA12A98
:1004A000A501A4002408A2052508A305A12AA501E9
:1004B000A4006F225D2AA501A40022308400240834
:1004C00080072508840F00000318013E031C8007E5
:1004D000A12AA309A209A20A0319A30A08007422E7
:1004E000A40A0319A50AA12AA509A409A12AA501FC
:1004F000A40086220139A12AA501A400862202397E
:10050000A12AA501A40086220439A12A25082302D4
:10051000031D8E2A2408220203190234031C04340A
:100520000134A301A200A12A0D20A9000005841B0B
:10053000290603190034013421200D20A6000408E7
:08054000A7008312640008000B
:084000007F007F007F007F00BC
:04400E00F53F010079
:00000001FF
